:020000000134C9
:20003400758176758901D2AFD28C1204C212001B80FB0581740A75F000C0E0C0F07402753E
:20005400F000C0E0C0F01207D215811581158115815480C5F05400C5F078FE122918F64573
:20007400F07003020098E612294A7BFF122941122A4B45F0700302009574FF75F0FF02006F
:200094009D020048740175F000158122120046740A75F000C0E0C0F0740075F000C0E0C00F
:2000B400F0740175F000C0E0C0F01207FB7FFA122924221200467BFF7CFF122A4B45F0708B
:2000D400030200E074FF75F0FF020149740A75F000C0E0C0F0740075F000C0E0C0F07438FC
:2000F40075F000C0E0C0F01207FB7FFA122924120046740A75F000C0E0C0F0740075F000E7
:20011400C0E0C0F0740C75F000C0E0C0F01207FB7FFA1229241200A0740075F000C0E0C06F
:20013400F0740075F000C0E0C0F012014A15811581158115812212004678FB122918E612A5
:20015400294A90020C022953740A75F000C0E0C0F0740075F000C0E0C0F078F5122918E6FA
:20017400248012294AC0E0C0F01207FB7FFA122924020220740A75F000C0E0C0F0740075C6
:20019400F000C0E0C0F078F5122918E624C012294AC0E0C0F01207FB7FFA1229240202209C
:2001B400740A75F000C0E0C0F0740075F000C0E0C0F078F5122918E6249412294AC0E0C08C
:2001D400F01207FB7FFA122924020220740A75F000C0E0C0F0740075F000C0E0C0F078F542
:2001F400122918E624D412294AC0E0C0F01207FB7FFA122924020220E0010300B40102003A
:20021400880101005C01000000002002220581740078FE122918F678FE122918E6181818EF
:2002340018860108860275F00012293A89828A83E49312294A7B00122941122A5445F07061
:20025400030202A7800B78FE122918E604F61480C6120046740A75F000C0E0C0F0740175D9
:20027400F000C0E0C0F078FA122918E618181818860108860275F00012293A89828A83E432
:200294009312294AC0E0C0F01207FB7FFA12292402025A78FA122918E60886F015812212A5
:2002B4000046740A75F000C0E0C0F0740175F000C0E0C0F078F7122918E612294AC0E0C0FA
:2002D400F01207FB7FFA122924227F0812292478F3122918E60886F07B007C00122A2B4561
:2002F400F0700302030D740075F00079F712291D12293A742DF702031D740075F00079F75C
:2003140012291D12293A742BF778F3122918E60886F078FD122918F608A6F078F31229182A
:20033400E60886F07B007C00122A2B45F0700302036B78FD122918E60886F0122A2478F3D8
:20035400122918F608A6F018E60886F0122A1118F608A6F0122A1A740175F00079F7122952
:200374001D12293A78F3122918E60886F07BE87C031229972430C5F03400C5F0F718E60812
:2003940086F07BE87C0312299078FD122918F608A6F0740275F00079F712291D12293A783A
:2003B400FD122918E60886F07B647C001229972430C5F03400C5F0F778F3122918E608862D
:2003D400F07B647C0012299078FD122918F608A6F0740375F00079F712291D12293A78FD09
:2003F400122918E60886F07B0A7C001229972430C5F03400C5F0F7740475F00079F71229EE
:200414001D12293A78FD122918E60886F07B0A7C001229902430C5F03400C5F0F77400756C
:20043400F00079F712291D12293AE712294AC0E0C0F01202B315811581740175F00079F782
:2004540012291D12293AE712294AC0E0C0F01202B315811581740275F00079F712291D1257
:20047400293AE712294AC0E0C0F01202B315811581740375F00079F712291D12293AE71244
:20049400294AC0E0C0F01202B315811581740475F00079F712291D12293AE712294AC0E06C
:2004B400C0F01202B3158115817FF8022933758E037481F5A8E5884401F5887400F53E74CE
:2004D40000F571740C75F000C0E0C0F0740075F000C0E0C0F0E53E12294AC0E0C0F0120733
:2004F400FB7FFA122924740075F000F53A85F03BF53885F0397400F5677400F511747075DF
:20051400F017F56185F062746475F000F55785F05879687A00E98AF0C0E0C0F0746475F0F2
:2005340000C0E0C0F012271D1581158115811581121A031200C7744B75F02EC0E0C0F012ED
:20055400022115811581740075F000C0E0C0F0740175F000C0E0C0F012014A158115811547
:20057400811581745475F02EC0E0C0F01202211581158174E875F003C0E0C0F01227501592
:2005940081158174BFF537E5114402F511121608748075F025C0E0C0F012276D15811581BF
:2005B40079B37A2AE98AF0C0E0C0F0122790158115811211431212361211A5121122120FC1
:2005D400FB1209C5120F26120C8E120D06120D4C1213081215331216DE121B1A1218E112B8
:2005F4001BB1121BDA121C98121EFD12234412099C12156C1215D612160812078E120FD297
:0A06140012242E1224A20205C922AE
:07000300C0D0C0E002061EA0
:20061E00C0F0C083C082C000C001C002C003C004C005C006C007120652D007D006D005D0AF
:20063E0004D003D002D001D000D082D083D0F0D0E0D0D032740875F000C0E0C0F07402754F
:20065E00F000C0E0C0F01207D21581158115811581F54185F042740875F000C0E0C0F07467
:20067E000175F000C0E0C0F01207D21581158115811581F54385F044E5438544F05410C568
:20069E00F05400C5F0F53FE5438544F05420C5F05400C5F0F540E5438544F0540FC5F0547A
:2006BE0000C5F0F54385F044E5438544F07B087C001229F2F54385F044E5418542F0454313
:2006DE00C5F04544C5F0F54185F042E53F6003020701E5418542F07BFF7CFF12297CF541CC
:2006FE0085F042E5407003020712740F75F027F54185F042E53E12294AC333C5F033C5F03B
:20071E0079477A0012293AE5418542F0F709A7F0E53E04F53E14E53E5403F53E740C75F098
:20073E0000C0E0C0F0740075F000C0E0C0F0E53E12294AC0E0C0F01207FB7FFA12292474CA
:20075E000175F000C0E0C0F012275015811581E53E12294A7B00122941122A4B45F0700342
:20077E0002078DE59054BFF590E5114480F51122E51675F0007B627C00122A4B45F07003EE
:20079E000207B679C67A2DE98AF0C0E0C0F0122790158115811211432278FB122918E6F5C5
:2007BE0013E513A2E09290A2E19291A2E29292A2E392932278F9122918E612294AC0E0C0C3
:2007DE00F01207B71581158178FB122918E60886F0C0E0C0F01227CC158115812278F712C1
:2007FE002918E612294AC0E0C0F01207B71581158178F9122918E60886F0C0E0C0F008E67D
:20081E0012294AC0E0C0F01227ED15811581158115812212280D74D075F000C0E0C0F012F3
:20083E00282215811581740775F000C0E0C0F012282215811581749075F000C0E0C0F012A1
:20085E0028221581158112281A2212280D74D075F000C0E0C0F012282215811581740075DD
:20087E00F000C0E0C0F01228221581158112281A12280D74D175F000C0E0C0F0122822158C
:20089E008115817400F5767400F515E51575F0007B067C00122A5E45F070030208E18008B5
:2008BE00E51504F5151480E3E515794F7A0075F00012293AC001C00212284CD007D000F6DF
:2008DE000208BE7401F576E515794F7A0075F00012293AC001C00212284CD007D000F61284
:2008FE00281A2212280D74D075F000C0E0C0F012282215811581740075F000C0E0C0F01273
:20091E00282215811581740075F000C0E0C0F012282215811581743075F000C0E0C0F01227
:20093E00282215811581741275F000C0E0C0F012282215811581740375F000C0E0C0F01222
:20095E00282215811581742575F000C0E0C0F012282215811581740775F000C0E0C0F012EB
:20097E00282215811581740075F000C0E0C0F01228221581158112281A2212086822E5161D
:20099E0075F0007B757C00122A4B45F070030209C479E37A2CE98AF0C0E0C0F012279015D7
:2009BE0081158112114322E51675F0007B747C00122A4B45F07003020A70745C75F02EC0E1
:2009DE00E0C0F012279015811581120B27F50D743A75F000C0E0C0F01227A41581158112B0
:2009FE000B27F50C743A75F000C0E0C0F01227A415811581120B27F50A12280D74D075F007
:200A1E0000C0E0C0F012282215811581740075F000C0E0C0F012282215811581E50A75F0DB
:200A3E0000C0E0C0F012282215811581E50C75F000C0E0C0F012282215811581E50D75F03B
:200A5E0000C0E0C0F01228221581158112281A121143227F09122924740075F00078FD127D
:200A7E002918F608A6F01227BCC0E0C0F01227A41581158178FC122918F67B0D7C00122A38
:200A9E005445F07003020AD9801678FD122918E60886F0122A1118F608A6F0122A1A80C600
:200ABE0078FD122918E60886F079F612291D12293A78FC122918E6F7020AA878FD12291890
:200ADE00E60886F079F612291D12293A7400F778FD122918E60886F07B007C00122A4B45FE
:200AFE00F07003020B0C74FF75F0FF020B2279F612291DE98AF0C0E0C0F012288015811577
:200B1E0081020B227FF702293305810581058105810581740075F00078FD122918F608A650
:200B3E00F078FD122918E60886F07B027C00122A2B45F07003020B99801678FD122918E689
:200B5E000886F0122A1118F608A6F0122A1A80D178FD122918E60886F079FA12291D122927
:200B7E003AC001C0021227BCC0E0C0F01227A415811581D007D000F6020B5878FD12291882
:200B9E00E60886F079FA12291D12293A7400F7740075F00079FA12291D12293AE7C39430A1
:200BBE0012294A7B041229411229F2C0E0C0F0740175F00079F812291D12293AE7C3943094
:200BDE00D004D0034BC5F04CC5F012294A7FFB02293305810581058105810581740075F07B
:200BFE000078FD122918F608A6F078FD122918E60886F07B027C00122A2B45F07003020C39
:200C1E0062801678FD122918E60886F0122A1118F608A6F0122A1A80D178FD122918E6083C
:200C3E0086F079FA12291D12293AC001C0021227BCC0E0C0F01227A415811581D007D00068
:200C5E00F6020C2178FD122918E60886F079FA12291D12293A7400F779FA12291DE98AF04C
:200C7E00C0E0C0F0122880158115817FFB022933E51675F0007B697C00122A4B45F0700359
:200C9E00020D05747B75F02EC0E0C0F012279015811581740075F000C0E0C0F01207B7154D
:200CBE00811581740475F000C0E0C0F0120A717B647C0012297CC0E0C0F01227FB15811504
:200CDE008115811581740475F000C0E0C0F01227DB15811581F56185F062E5618562F0F59D
:200CFE005F85F06012114322E51154087003020D4BE55F8560F0122A1AF55F85F060122A27
:200D1E0011E55F8560F07B007C00122A6545F07003020D4BE5618562F0F55F85F060E511B5
:200D3E004404F5111222D4E51154DFF511220581E51714F51704E51775F0007B007C0012DE
:200D5E002A6545F07003020F237464F517120868740275F000794F7A0012293AE775F000C6
:200D7E007B047C00122A0078FE122918F6E675F0007B0A7C0012297CF6740275F000794FC3
:200D9E007A0012293AC001C002740275F000794F7A0012293AE7540F78FC12291826D00723
:200DBE00D000F6740175F000794F7A0012293AE775F0007B047C00122A0078FE122918F67C
:200DDE00E675F0007B0A7C0012297CF6740175F000794F7A0012293AC001C002740175F00E
:200DFE0000794F7A0012293AE7540F78FC12291826D007D000F6740075F000C0E0C0F0120F
:200E1E0007B715811581740275F000794F7A0012293AC001C002740075F000C0E0C0F0127A
:200E3E0027CC15811581D007D00086037C00122A4B45F0602B740175F000794F7A0012292B
:200E5E003AC001C002740175F000C0E0C0F01227CC15811581D007D00086037C00122A4B29
:200E7E0045F07003020EB2E5114408F511742C75F001F55785F058743D75F000C0E0C0F01D
:200E9E00E51175F000C0E0C0F01227ED1581158115811581740275F000794F7A0012293A79
:200EBE00C001C002740275F000C0E0C0F01227CC15811581D007D00086037C00122A4B45BD
:200EDE00F0602B740175F000794F7A0012293AC001C002740375F000C0E0C0F01227CC151F
:200EFE00811581D007D00086037C00122A4B45F07003020F23E51154F7F511746475F0002A
:200F1E00F55785F058158122E51675F0007B647C00122A4B45F07003020FD1749375F02E7C
:200F3E00C0E0C0F012279015811581120B27F50E742D75F000C0E0C0F01227A415811581A8
:200F5E00120B27F50F742D75F000C0E0C0F01227A415811581120B27F51012280D74D07583
:200F7E00F000C0E0C0F012282215811581740475F000C0E0C0F012282215811581E50E756E
:200F9E00F000C0E0C0F012282215811581E50F75F000C0E0C0F012282215811581E51075D0
:200FBE00F000C0E0C0F01228221581158112281A12114322E51675F0007B0D7C00122A4B84
:200FDE0045F07003020FFA79B37A2AE98AF0C0E0C0F01227901581158112114322E51675D0
:200FFE00F0007B2F7C00122A4B45F0700302112112086874B275F02EC0E0C0F0740475F0F2
:20101E0000794F7A0012293AE775F000C0E0C0F0740575F000794F7A0012293AE775F0007E
:20103E00C0E0C0F0740675F000794F7A0012293AE775F000C0E0C0F0740475F0001224D924
:20105E007FF812292474C375F02EC0E0C0F0740275F000794F7A0012293AE775F000C0E004
:20107E00C0F0740175F000794F7A0012293AE775F000C0E0C0F0740075F000794F7A001248
:20109E00293AE775F000C0E0C0F0740475F0001224D97FF812292412121174D375F02EC0A2
:2010BE00E0C0F0740075F00079477A0012293AE70987F0C0E0C0F0740275F00079477A002E
:2010DE0012293AE70987F0C0E0C0F0740475F00079477A0012293AE70987F0C0E0C0F0740F
:2010FE000675F00079477A0012293AE70987F0C0E0C0F0740575F0001224D97FF612292440
:20111E0012114322E5985401700302113E1227BCC0E0C0F01227A415811581F516021142E5
:20113E0074FFF5162279CE7A2AE98AF0C0E0C0F0122790158115812205810581740075F057
:20115E000078FD122918F608A6F078FD122918E60886F078F91229188603088604122A2BA3
:20117E0045F070030211A0801678FD122918E60886F0122A1118F608A6F0122A1A80CB0298
:20119E00118715811581221211AC1211E622E55D855EF0122A11F55D85F05E122A1AE55D32
:2011BE00855EF0AB57AC58122A6E45F070030211E5740075F000F55D85F05EE5114440F581
:2011DE0011C2977405F51422E51154407003021210E51414F51404E51475F0007B007C0053
:2011FE00122A4B45F07003021210D297E51154BFF51122E5904440F590E511548075F00037
:20121E007B007C00122A4B45F0700302122F021217E511547FF51122308DFDC28D438CDC77
:20123E002205810581740175F00079687A0012293AE775F00078FD122918F608A6F018E612
:20125E000886F07B087C001229F218F608A6F0740075F00079687A0012293A78FD122918A9
:20127E00E60886F047158115812274012568F568E43569F569E4356AF56A221212887402F2
:20129E0075F00079687A0012293AE775F000C0E0C0F01207B71581158112123F2212128832
:2012BE00121288740275F00079687A0012293AE775F000C0E0C0F01207B7158115811212FD
:2012DE003F2278FB122918E675F0007B047C00122A00F62430C5F03400C5F02278FB12298F
:2012FE0018E6540F243012294A22E511540470030214F11212111208681212BBC0E0C0F0C6
:20131E00E55B855CF0C0E0C0F01227FB1581158115811581121299C0E0C0F0740475F000D8
:20133E00794F7A0012293AE775F000C0E0C0F01227ED1581158115811581121299C0E0C0A1
:20135E00F0740575F000794F7A0012293AE775F000C0E0C0F01227ED1581158115811581D0
:20137E00121299C0E0C0F0740675F000794F7A0012293AE775F000C0E0C0F01227ED158154
:20139E00158115811581121299C0E0C0F0740275F000794F7A0012293AE775F000C0E0C022
:2013BE00F01227ED1581158115811581121299C0E0C0F0740175F000794F7A0012293AE71C
:2013DE0075F000C0E0C0F01227ED1581158115811581121299C0E0C0F0740075F000794F0E
:2013FE007A0012293AE775F000C0E0C0F01227ED15811581158115811212BBC0E0C0F07423
:20141E000075F00079477A0012293AE70987F0C0E0C0F01227FB1581158115811581121233
:20143E00BBC0E0C0F0740275F00079477A0012293AE70987F0C0E0C0F01227FB15811581E2
:20145E00158115811212BBC0E0C0F0740475F00079477A0012293AE70987F0C0E0C0F012BE
:20147E0027FB15811581158115811212BBC0E0C0F0740675F00079477A0012293AE70987A0
:20149E00F0C0E0C0F01227FB1581158115811581E51154FBF511E55B855CF0122A11F55B69
:2014BE0085F05C1214F2740075F000C0E0C0F01207B715811581740675F000C0E0C0F0E5EC
:2014DE005B855CF0C0E0C0F01227FB158115811581158122E55B855CF07B887C13122A6E77
:2014FE0045F07003021532E51154F7F511746475F000F55785F058743C75F000C0E0C0F0DB
:20151E0074FF75F0FFC0E0C0F01227ED158115811581158122E51675F0007B727C00122AE1
:20153E004B45F0700302156B74E075F02EC0E0C0F0E55B855CF0C0E0C0F0740275F0001293
:20155E0024D9158115811581158112114322740E75F000C0E0C0F0740075F000C0E0C0F030
:20157E001207D215811581158115817BFF7C00122A5445F0600EE511540175F0007B007C3A
:20159E0000122A4B45F070030215D1E5114401F511740E75F000C0E0C0F0740075F000C005
:2015BE00E0C0F01207D21581158115811581F5370215D574FFF53722740E75F000C0E0C01A
:2015DE00F0740075F000C0E0C0F01207D215811581158115817BFF7C00122A4B45F070036C
:2015FE00021607E51154FEF51122E53775F0007BFF7C00122A5445F070030216DDE5377509
:20161E00F0009016C9022953E57104F571140216DDE5116402F511E51154EFF5111200A0B3
:20163E00740075F000C0E0C0F0740175F000C0E0C0F012014A158115811581158174F675A5
:20165E00F02EC0E0C0F012022115811581E51154027003021687742A75F000C0E0C0F012DA
:20167E0002B3158115810216C01200A01223A2740075F000C0E0C0F0740075F000C0E0C0A8
:20169E00F012014A158115811581158174FE75F02EC0E0C0F012022115811581E511441087
:2016BE00F5110216DD0216DD0216DDC616EF00C316DF002F16BF0026167F000000DD1622D0
:2016DE00E51675F0007B737C00122A4B45F07003021884740075F000C0E0C0F01207B71547
:2016FE00811581740775F02FC0E0C0F0740075F000C0E0C0F01227CC15811581C0E0C0F0AC
:20171E00740175F000C0E0C0F01227CC15811581C0E0C0F0740375F0001224D97FFA122961
:20173E0024740075F000C0E0C0F0120BF012294AC0E0C0F01227ED1581158115811581746A
:20175E003A75F000C0E0C0F01227A415811581740175F000C0E0C0F0120BF012294AC0E017
:20177E00C0F01227ED1581158115811581741A75F02FC0E0C0F0740275F000C0E0C0F0126E
:20179E0027CC15811581C0E0C0F0740375F000C0E0C0F01227CC15811581C0E0C0F0740398
:2017BE0075F0001224D97FFA122924740275F000C0E0C0F0120BF012294AC0E0C0F0122779
:2017DE00ED1581158115811581743A75F000C0E0C0F01227A415811581740375F000C0E0BE
:2017FE00C0F0120BF012294AC0E0C0F01227ED1581158115811581742D75F02FC0E0C0F036
:20181E00740075F000C0E0C0F01227CC15811581C0E0C0F0740175F000C0E0C0F01227CCD1
:20183E0015811581C0E0C0F0740275F000C0E0C0F01227CC15811581C0E0C0F0740375F086
:20185E0000C0E0C0F01227CC15811581C0E0C0F0740575F0001224D97FF612292412188529
:20187E001223A212114322740075F000C0E0C0F01227CC158115817B637C00122A4B45F07B
:20189E0070030218C3743C75F000C0E0C0F0740175F000C0E0C0F01227ED15811581158163
:2018BE0015810218E0743C75F000C0E0C0F074FF75F0FFC0E0C0F01227ED15811581158106
:2018DE00158122E51675F0007B3D7C00122A4B45F07003021A02740075F000C0E0C0F01216
:2018FE0007B715811581744375F02FC0E0C0F0740075F000C0E0C0F01227CC15811581C02B
:20191E00E0C0F0740175F000C0E0C0F01227CC15811581C0E0C0F0740375F0001224D97F04
:20193E00FA122924745575F02FC0E0C0F0740275F000C0E0C0F01227CC15811581C0E0C0C7
:20195E00F0740375F000C0E0C0F01227CC15811581C0E0C0F0740375F0001224D97FFA1256
:20197E002924746775F02FC0E0C0F0740475F000C0E0C0F01227DB158115817B647C001263
:20199E002997C0E0C0F0740275F0001224D91581158115811581743C75F000C0E0C0F01260
:2019BE0027CC158115817B017C00122A4B45F070030219EA748575F02FC0E0C0F0740175F7
:2019DE00F0001224D9158115810219FF748E75F02FC0E0C0F0740175F0001224D91581152A
:2019FE008112114322740075F000C0E0C0F01207B715811581743D75F000C0E0C0F01227FC
:201A1E00CC15811581F511740475F000C0E0C0F01227DB15811581F56185F062E5618562E3
:201A3E00F0F55F85F060740675F000C0E0C0F01227DB15811581F55B85F05C796E7A00E995
:201A5E008AF0C0E0C0F0742E75F000C0E0C0F012271D1581158115811581796B7A00E98AC8
:201A7E00F0C0E0C0F0E55B855CF0C0E0C0F012271D1581158115811581796B7A00E98AF038
:201A9E00C0E0C0F0796E7A00E98AF0C0E0C0F012266F1581158115811581796B7A00E98AF4
:201ABE00F0C0E0C0F0746475F000C0E0C0F012271D158115811581158179727A00E98AF0C5
:201ADE00C0E0C0F0796B7A00E98AF0C0E0C0F012262E158115811581158179687A00E98AFB
:201AFE00F0C0E0C0F079727A00E98AF0C0E0C0F01226E0158115811581158122E51675F07E
:201B1E00007B6E7C00122A4B45F07003021BB0749575F02FC0E0C0F0122790158115811252
:201B3E0027BC7B797C00122A4B45F07003021BADE51154F7F511740075F000F55B85F05CFA
:201B5E00740075F000C0E0C0F01207B715811581740675F000C0E0C0F0740075F000C0E09A
:201B7E00C0F01227FB158115811581158179687A00E98AF0C0E0C0F0746475F000C0E0C060
:201B9E00F012271D158115811581158112216A12114322E51675F0007B3F7C00122A4B4502
:201BBE00F07003021BD979D27A2AE98AF0C0E0C0F01227901581158112114322E51675F02F
:201BDE00007B637C00122A4B45F07003021C9712086874A875F02FC0E0C0F0740475F0004A
:201BFE00794F7A0012293AE775F000C0E0C0F0740575F000794F7A0012293AE775F000C0D3
:201C1E00E0C0F0740675F000794F7A0012293AE775F000C0E0C0F0740475F0001224D97F79
:201C3E00F812292474B975F02FC0E0C0F0740275F000794F7A0012293AE775F000C0E0C0E0
:201C5E00F0740175F000794F7A0012293AE775F000C0E0C0F0740075F000794F7A001229F3
:201C7E003AE775F000C0E0C0F0740475F0001224D97FF812292412114322E51675F0007B4B
:201C9E00617C00122A4B45F07003021EFC12223E796B7A00E98AF0C0E0C0F0740175F000A1
:201CBE00C0E0C0F012271D158115811581158179687A00E98AF0C0E0C0F0796B7A00E98A29
:201CDE00F0C0E0C0F01226411581158115811581796B7A00E98AF0C0E0C0F079687A00E980
:201CFE008AF0C0E0C0F01226E0158115811581158179687A00E98AF0C0E0C0F0746475F041
:201D1E0000C0E0C0F012271D1581158115811581740075F000F56585F066E5658566F0ABC9
:201D3E005BAC5C122A5E45F07003021EF98012E5658566F0122A11F56585F066122A1A80B8
:201D5E00D9740D75F000C0E0C0F012215815811581740A75F000C0E0C0F012215815811536
:201D7E00811212BBC0E0C0F01227DB1581158174C975F02FC0E0C0F0E5658566F0C0E0C0AF
:201D9E00F0740275F0001224D9158115811581158174CD75F02FC0E0C0F0121299C0E0C0B1
:201DBE00F01227CC15811581C0E0C0F0121299C0E0C0F01227CC15811581C0E0C0F01212E2
:201DDE0099C0E0C0F01227CC15811581C0E0C0F0740475F0001224D97FF812292474DD75F3
:201DFE00F02FC0E0C0F0121299C0E0C0F01227CC15811581C0E0C0F0121299C0E0C0F012A9
:201E1E0027CC15811581C0E0C0F0121299C0E0C0F01227CC15811581C0E0C0F0740475F0CA
:201E3E00001224D97FF812292474ED75F02FC0E0C0F01212BBC0E0C0F01227DB15811581EB
:201E5E00C0E0C0F0740275F0001224D9158115811581158174F175F02FC0E0C0F01212BBAA
:201E7E00C0E0C0F01227DB15811581C0E0C0F0740275F0001224D9158115811581158174AE
:201E9E00F575F02FC0E0C0F01212BBC0E0C0F01227DB15811581C0E0C0F0740275F000129F
:201EBE0024D9158115811581158174F975F02FC0E0C0F01212BBC0E0C0F01227DB15811570
:201EDE0081C0E0C0F0740275F0001224D9158115811581158112211E021D4D12114322E5A7
:201EFE001675F0007B787C00122A4B45F0700302211D12223E796B7A00E98AF0C0E0C0F0E8
:201F1E00740175F000C0E0C0F012271D158115811581158179687A00E98AF0C0E0C0F07944
:201F3E006B7A00E98AF0C0E0C0F01226411581158115811581796B7A00E98AF0C0E0C0F009
:201F5E0079687A00E98AF0C0E0C0F01226E0158115811581158179687A00E98AF0C0E0C0C7
:201F7E00F0746475F000C0E0C0F012271D1581158115811581740075F000F56585F066E525
:201F9E00658566F0AB5BAC5C122A5E45F0700302211A8012E5658566F0122A11F56585F083
:201FBE0066122A1A80D9740D75F000C0E0C0F012215815811581740A75F000C0E0C0F012BC
:201FDE002158158115811212BBC0E0C0F01227DB1581158174FD75F02FC0E0C0F0E56585AB
:201FFE0066F0C0E0C0F0740275F0001224D91581158115811581121299C0E0C0F01227CCC9
:20201E0015811581121299C0E0C0F01227CC15811581121299C0E0C0F01227CC15811581FA
:20203E00121299C0E0C0F01227CC15811581121299C0E0C0F01227CC15811581121299C089
:20205E00E0C0F01227CC15811581740175F030C0E0C0F01212BBC0E0C0F01227DB15811559
:20207E0081C0E0C0F0740275F0001224D91581158115811581740575F030C0E0C0F01212AD
:20209E00BBC0E0C0F01227DB15811581C0E0C0F0740275F0001224D9158115811581158145
:2020BE00740975F030C0E0C0F01212BBC0E0C0F01227DB15811581C0E0C0F0740275F00006
:2020DE001224D91581158115811581740D75F030C0E0C0F01212BBC0E0C0F01227DB15813C
:2020FE001581C0E0C0F0740275F0001224D9158115811581158112211E021FB212114322EE
:20211E0005811228C47B137C00122A4B45F0700302215578FE122918E612294A7B11122971
:20213E0041122A5445F070030221551228C478FE122918F602213115812278FB122918E61B
:20215E00F5133099FDC299E513F59922741175F030C0E0C0F01227901581158179187A0026
:20217E00E98AF0C0E0C0F0741E75F000C0E0C0F01228D61581158115811581740075F00006
:20219E00C0E0C0F01207B715811581740075F000F56585F066E5658566F079187A0012295C
:2021BE003AE775F0007B007C00122A5445F070030222188012E5658566F0122A11F565852D
:2021DE00F066122A1A80CEE5658566F02408C5F03400C5F0C0E0C0F0E5658566F079187A78
:2021FE000012293AE775F000C0E0C0F01227ED15811581158115810221D3E5658566F024F3
:20221E0008C5F03400C5F0C0E0C0F0740075F000C0E0C0F01227ED158115811581158122E1
:20223E000581740D75F000C0E0C0F012215815811581740A75F000C0E0C0F01221581581B9
:20225E001581740075F000C0E0C0F01207B715811581740075F000F56585F066E565856662
:20227E00F02408C5F03400C5F0C0E0C0F01227CC1581158178FE122918F67B007C00122A13
:20229E005445F070030222D18012E5658566F0122A11F56585F066122A1A80C078FE1229AF
:2022BE0018E612294AC0E0C0F01227A4158115810222A8158122E51154F7F511746475F01C
:2022DE0000F55785F05822E56704F56712294A7B32122941122A3B45F0700302233B740058
:2022FE00F567E53A853BF0F53885F039E5B054087003022320740175F000F53A85F03B0256
:20231E00232A740075F000F53A85F03BE53A853BF0C39538C5F09539C5F0022343740075B2
:20233E00F00002234322740075F000C0E0C0F01207B715811581743C75F000C0E0C0F01269
:20235E0027CC158115817B017C00122A4B45F070030223A11222E512294A7B0012294112AC
:20237E002A2B45F070030223A1E5114408F511E5618562F0F55F85F060742C75F001F5579C
:20239E0085F05822740075F000C0E0C0F01207B715811581743C75F000C0E0C0F01227CCA1
:2023BE00158115817B017C00122A4B45F07003022400740775F000C0E0C0F0740175F0007C
:2023DE00C0E0C0F012014A1581158115811581744D75F000C0E0C0F01202B315811581026F
:2023FE00242D740775F000C0E0C0F0740175F000C0E0C0F012014A158115811581158174EB
:20241E004175F000C0E0C0F01202B31581158122E511540270030224A1121211740075F0FF
:20243E0000C0E0C0F0740075F000C0E0C0F012014A1581158115811581E5715403F571E558
:20245E0071243175F000C0E0C0F01202B315811581742075F000C0E0C0F01202B315811535
:20247E0081E57175F000C333C5F033C5F079477A0012293AE70987F0C0E0C0F01202DE1502
:20249E0081158122E511541070030224D8740075F000C0E0C0F0740175F000C0E0C0F012B5
:2024BE00014A1581158115811581E55B855CF0C0E0C0F01202DE158115812223F42581F805
:2024DE00868208868308E4FEFF93700122B42555A3E493B42D06430780A3E493B430034379
:2024FE00074024D0B40A00500CCE75F00AA42EFEA3E49380EDE493B46413E60886F030F7A8
:20251E0008430720122A21A6F018F68003B4750543070A801CB478054307108014B46F0B3C
:20253E00430708800C1227AAA3809BB462624307027A00C004C005C006C007AB0753031F83
:20255E007C00E60886F01229BFA6F018F6EDD007D006D005D0042430B43A0040022407C02D
:20257E00E00AE645F070CCA902EF30E506742D1227AA0A12260FD0E01227AAD9F90808EF0E
:20259E0030E7A5EAC39E50A074201227AA0A80F3B4630BAA0112260FE61227AA80DFB473CF
:2025BE002BC082C08386820886837A00E4936004A30A80F8868318868212260FE493A360D0
:2025DE00051227AA80F6D083D08280B1B4691986017A00E76004090A80F912260F8601E7E6
:2025FE00609B1227AA0980F7F97A0112260FE980A8EE601B8FF020F716C002EAC39E500D14
:20261E00742030F60274301227AA0A80EED0022212273A7A04C3E637F60809DAF9E4F5F079
:20263E0092E02212273A7A04C3E697F60809DAF980EB122732C37A04E633F608DAFA80DD7E
:20265E001227327A04C82AC8C318E613F6DAFA80CC12273AAB00A8817F0412292408AC00F2
:20267E001226E3122746A80312266150077872A904122631A8031226EF600CA80412265392
:20269E00A8041226EF70DFA80379721226E37FFC02293312273AAB00AC011227467D21C3C5
:2026BE00A803122654DD02803378721226547872A9041226FE20E7E77872A904122644D31C
:2026DE0080DE12273A7A04E7F60908DAFA221227327A0475F000E6700308DAFA2212273A91
:2026FE007A04E82AF8E92AF9181987F0E6B5F006DAF6E4F5F02274FF40F904F5F00422E594
:20271E008124FBF9870012274887000909E7F60809E7F622E58124FBF8860022E58124FBCA
:20273E00F88601181886002278727A04760008DAFB2278FB1229188603088604BB0004BCEB
:20275E0000012279E5A3D9FD1BBBFFF01C80F478FB1229188603088604748075F070122927
:20277E00BF122A21758921F58DF58B7588597598522278FB1229188682088683E493602D44
:20279E001227AAA380F678FB122918E63099FDC299F599B40A17740D80F2E430980C30987C
:2027BE00FDC298E599B40D02740A75F0002278FB1229188682088683E075F0002278FB1293
:2027DE0029188682088683E0F5F0A3E0C5F02278F9122918868208868308E6F02278F91202
:2027FE002918868208868308E608F0A3E6F022D295122872C295122878C29422C2951228BB
:20281E0072D2952278FB122918E67F0830E704D2958002C29512287223C294DFEFD29512A5
:20283E002872309500122878C294122878227F087400D295122872A29533C294DFF6C0E0FC
:20285E00D295E576B40002C295122872C294D0E075F00022D2943094FD22000022000000E7
:20287E00002278FB1229188601E4FBFCFFE709B42D030FE709C39430B40A005012FA740AFF
:20289E0075F00012297C2AFBE5F03400FC80E4EB8CF0DF03022A212278FB122918E6309943
:2028BE00FDC299F5992274FFF5F030980A3098FDC298E59975F0002278FB1229188604183C
:2028DE00188601E4FD1227BCB408028003B47F16ED60F21D74081227AA74201227AA74082D
:2028FE001227AA1980DF1227AAF724F36006090DEDB504D1E4F7F5F0ED22C82581C822C98B
:20291E002581C97A0022D083D082CF2581F581CFC082C08322CF2581F581CF2229F9E5F0B5
:20293E003AFA227C00CB30E7011CCB2275F00030E70215F022FDE493A3FEE493A3FF4E702A
:20295E0009E493FE740193FF800BE493A3B5050BE493B5F0068F838E82E473A380D8FEEBEB
:20297E00A4FD8EF0ECA4FCEB8EF0A4C5F02C2DC5F0221229BF8EF0ED22C0F0C0E0E5F06C84
:20299E005480FF8CF030F707EB122A21ACF0FBD0E0D0F030F703122A21BF80051229BF8008
:2029BE0062C002C001AAF0F97E007D007F11C3E933F9EA33FADF08F5F0E9D001D00222EDA0
:2029DE0033FDEE33FEC3ED9BF5F0EE9C40E0ADF0FED380DBBB000122C333C5F033C5F0DB9B
:2029FE00F722BB000122C3C5F013C5F013DBF722122A1104700205F022122A1A14B4FF0282
:202A1E0015F022122A1AF4C5F0F4C5F022122A7E4029801E122A7E40227017801E122A7EEB
:202A3E0040107017800C122A7E50108005122A926009E4F5F022122A9260F7E4F5F0042240
:202A5E00122A9240F680EB122A9240EF70E480EB122A9240DD70E480D9122A9250DD80D248
:202A7E00C39BC5F09C20E70720D207C345F02220D2F9D322C5F0C39C7003E5F09B22FBE490
:202A9E0093CB22FCE493FB740193CC22FAE493F9740193CA220A0A4D696E694C4F474745C7
:202ABE00522056332E3020283F2068656C7029000A3E3E000A0A48454C50204D454E5520EE
:202ADE002020202020202020202020202020200A2F207072696E7420616E616C6F6720724E
:202AFE00656164696E67202020202020202020202020202020200A742054494D452073658B
:202B1E0074202020202020202020202020202020200A64204441544520736574202020208B
:202B3E002020202020202020202020200A6320436C6F636B20646973706C617920202020E8
:202B5E002020202020202020202020200A73207365742053544152542F53544F50207265D4
:202B7E00636F7264696E672074696D65202020202020202020202020202020200A6920737C
:202B9E00616D706C696E6720496E74657276616C20202020202020202020202020202020CA
:202BBE000A3D20646973706C61792073657474696E6720706172616D6574657273202020C8
:202BDE00202020202020202020202020200A72206E756D626572206F66207265636F72647E
:202BFE00202020202020202020202020202020200A62207465726D696E616C20636F6E6E01
:202C1E00656374696F6E202020202020202020202020202020200A6E204E657720726563F8
:202C3E006F7264202020202020202020202020202020200A6120414C4C20726561643A20B7
:202C5E0073616D706C65207265616C2D74696D6520616E6420646174612020202020202047
:202C7E002020202020202020200A78205265616420416C6C3A2073616D706C6520616E6490
:202C9E002064617461202020202020202020202020202020200A752041626F7574204D69EC
:202CBE006E694C4F474745522056332E30202020202020202020202020202020200A3F20EF
:202CDE0068656C70000A4D696E694C4F474745522077617320646573696E6765642062790D
:202CFE0020576963686974205349524943484F5445203238204A756E652032303033202003
:202D1E002020202020202020202020202020200A4170706C696564205068797369637320C9
:202D3E00446570742E204B4D49544C20202020202020202020202020202020200A666972AE
:202D5E006D7761726520757064617465643A203235204A756E652032303034202020202039
:202D7E002020202020202020202020200A55524C3A207777772E6B6D69746C2E61632E7416
:202D9E00682F7E6B7377696368697420656D61696C3A206B73776963686974406B6D6974BD
:202DBE006C2E61632E7468000A203120202020322020202033202020203420202020352044
:202DDE00202020362020202037202020203820202020392020203130202031312020313211
:202DFE0020202020202020202020202020202020202020200A494E312B20494E312D2049BA
:202E1E004E322B20494E322D20494E332B20494E332D20494E342B20494E342D202D3556A1
:202E3E00202B35562020305620202B56004D696E694C4F47470045522056332E30000A6554
:202E5E006E7465722063757272656E742074696D652048483A4D4D3A5353203E000A206954
:202E7E006E74657276616C20312D36303020736563203E20000A656E746572206375727247
:202E9E00656E7420646174652044442D4D4D2D5952203E000A253032782D253032782D25E3
:202EBE003032782000253032783A253032783A253032782000202564202564202564202529
:202EDE0064000A2575207265636F72647320617661696C61626C650078302E316D5620000F
:202EFE005265636F72643D20000A535441525420253032643A25303264203E000A53544FD2
:202F1E00502020253032643A25303264203E000A20253032643A2530326420253032643A16
:202F3E0025303264000A20535441525420253032643A25303264000A2053544F50202025CB
:202F5E003032643A25303264000A2053414D504C494E4720494E54455256414C28736563FB
:202F7E0029203D202575000A204D414E55414C000A204155544F000A204E657720726563FA
:202F9E006F72643F28592F4E29000A253032782D253032782D253032782000253032783AAE
:202FBE00253032783A2530327820002025640020253032782D253032782D2530327800205B
:202FDE00253032783A253032783A253032780020256400202564002025640020256400209E
:202FFE00256400202564002025640020256400202564000A3C2D2D20456E746572206465DF
:20301E00736372697074696F6E207465787420286D617820333020636861726163746572F4
:07303E0073292D2D3E0A004D
:00000001FF
